:100A9D0000C000F900A400B000990092008200F897
:100AAD00008000900088008300C600A10086008EA3
:060C4500EF13135401FF40
:0A0C4B00E51125E0F511EF4211223A
:0D0CAC00E51125E0F511EFF454014211228D
:040D9700EF521122E4
:070D5400EFF45401521122DB
:040D9B00EF421122F0
:070D5B00EFF45401421122E4
:0E0C7400E511F45401FFE51154FE4FF5112275
:060D8500E5115401FF22FC
:0D0CB900E511C313FFE51154015FF5112291
:0D0CC600E511C313FFE51154014FF5112294
:0E0C8200E51125E0F511EDF45F540142112259
:0E0C9000E51125E0F511EFF45D54014211224B
:08000300EDF45F5401521122DB
:080D3C00EFF45D540152112295
:080D4400EDF45F54014211229D
:080D4C00EFF45D540142112295
:070D6200EDF45F5401FF22D4
:070D6900EFF45D5401FF22CD
:0D0CD300E51825E0FFE51154014FF518224A
:0D0CE000E5185401FFE51154FE4FF51122F7
:100B5500E5185401FFE51154FE4FF511E518C313CF
:030B6500F518225E
:100C55008E5E8F5FE55F2DFFE55E3C8FF00206C27D
:100B68008E608F61C3E5619DFFE5609C8FF0020692
:010B7800C2BA
:090D3300120601EE8FF00206C267
:0F0C65008B5B8A5C895D120613EE8FF00206C26C
:070D7000E475F00102068AA0
:070D770074FFF5F002068A8B
:100B79008E628F63E5625CFFE5635DCF8FF00206ED
:010B8900C2A9
:100B8A008E648F65E5644CFFE5654DCF8FF00206F4
:010B9A00C298
:100B9B008E668F67E5666CFFE5676DCF8FF002069B
:010BAB00C287
:100BAC00EFF4FFEEF4FEEF2401FFE43E8FF00206BB
:010BBC00C276
:060D8B00EFF45401FF2209
:060D9100EE8FF00206C225
:0A0D2900EFF4FFEEF48FF00206C2B3
:100A47008B4B8A4C894D12065FFFAEF0AB4EAA4F17
:100A5700A95012065FFDAB4BAA4CA94DE5F08DF0EE
:0F0A67001206C2AB4EAA4FA950EE8FF00206C284
:100736008E528F538B548A5589567C037DE8120658
:1007460013EFC454F07B00FAAE52AF537C037DE83E
:100756001206138C528D53AE52AF537C007D641239
:100766000613EFFEE4EE4202AE52AF537C007D6408
:100776001206138C528D53AE52AF537C007D0A1273
:100786000613EFC4F8540FC868FFEEC454F048FED1
:10079600EFFBEE4202AE52AF537C007D0A12061307
:1007A6008C528D53E5524AFFE5534BAB54AA55A9DB
:0707B60056CF8FF00206C2CE
:10083C008E578F58E558780CCEA2E713CE13D8F804
:10084C007E00540FFF7C037DE81206018E598F5AEF
:10085C00E557FF3395E07E00EF540FFF7C007D647D
:10086C00120601EF255AF55AEE3559F559E558AEF1
:10087C00577804CEA2E713CE13D8F87E00540FFF9E
:10088C007C007D0A120601EF255AF55AEE3559F512
:10089C0059E558540F255AF55AE43559F559855AE6
:0408AC00F00206C28E
:100ABD00E51125E0F511C3EF9DEC6480F8EE64803F
:0B0ACD00984004431101225311FE2247
:100AD800E51125E0F511D3EF9DEC6480F8EE648014
:0B0AE800985004431101225311FE221C
:100AF300E51125E0F511D3EF9DEC6480F8EE6480F9
:0B0B0300984004431101225311FE2210
:100B0E00E51125E0F511C3EF9DEC6480F8EE6480ED
:0B0B1E00985004431101225311FE22E5
:100B2900E51125E0F511EF6D7002EE6C60044311DB
:060B390001225311FE220F
:100B3F00E51125E0F511EFB50508EEB504044311F5
:060B4F0001225311FE22F9
:100BBD00C3EF9DEC6480F8EE64809850035311FEF2
:010BCD002205
:100BCE00D3EF9DEC6480F8EE64809840035311FEE1
:010BDE0022F4
:100BDF00D3EF9DEC6480F8EE64809850035311FEC0
:010BEF0022E3
:100BF000C3EF9DEC6480F8EE64809840035311FECF
:010C000022D1
:0C0CED00EFB50507EEB504035311FE221D
:0C0CF900EF6D7002EE6C60035311FE22E0
:100C0100C3EF9DEC6480F8EE6480984003431101CA
:010C110022C0
:100C1200D3EF9DEC6480F8EE648098500343110199
:010C220022AF
:100C2300D3EF9DEC6480F8EE648098400343110198
:010C3300229E
:100C3400C3EF9DEC6480F8EE648098500343110187
:010C4400228D
:0C0D0500EF6D7002EE6C600343110122E0
:0C0D1100EFB50507EEB504034311012205
:070D7E00E4FF0FBF0AFC2295
:100A1700E4FEC2B4120D7EC2B3120D7ED2B3120D24
:100A27007ED2B4120D7EE4FDEE25E0FE3094034342
:100A37000601C2B3120D7ED2B30DBD08EBAF06227D
:100420000510E510C394054003E4F510E5101460D1
:100430005B1470030204DC147003020528240360BB
:100440000302057A7C0090000DE0540FFD25E0FFCB
:10045000EC33FE749D2FF582740A3EF583E493FC21
:10046000740193FD43040890010AE0FFC4131313C1
:10047000540130E0057DFF0205D0EF131313541F24
:1004800020E0030205D053057F0205D090000CE068
:10049000FEA3E07804CEA2E713CE13D8F87C005474
:1004A0000FFD25E0FFEC33FE749D2FF582740A3EAC
:1004B000F583E493FC740193FD43040490010BE085
:1004C00030E0057DFF0205D090010AE0FFC4540F23
:1004D00020E0030205D053057F0205D090000CE018
:1004E000FF3395E07C00EF540FFD25E0FFEC33FE79
:1004F000749D2FF582740A3EF583E493FC74019396
:10050000FD43040290010BE0FFC31330E0057DFFC3
:100510000205D090010AE0FFC413540720E0030253
:1005200005D053057F0205D090000CE0FEA3E078D3
:100530000CCEA2E713CE13D8F87C00540FFD25E0B3
:10054000FFEC33FE749D2FF582740A3EF583E4932D
:10055000FC740193FD43040190010BE0FF1313545D
:100560003F30E0047DFF806890010AE0FFC4131370
:10057000540330E05B53057F805690010BE0F9C4D3
:100580001313540175F008A4FBAAF0E9C413131364
:10059000540175F010A4FFE5F04AFAEF4BFBE9C4F3
:1005A00013540175F004A4FFEA45F0FAEB4FFBE9A0
:1005B000C4540125E0FFE4334AFEEB4FFFE9131377
:1005C000135401FBEEEF4BF4FFEEF47410FCAD0797
:1005D0007B10C2B3120D7EEC20E704C2B78002D2BA
:1005E000B7120D7EED25E0FDEC33FCD2B3120D7E8B
:1005F000DBE0D2B7120D7EC2B5120D7ED2B5020D70
:010600007E7B
:10023A00E52E700302041F152E0517E517B40517DE
:10024A00AF30EFC4135401F45401FFC43354E0FF38
:10025A00E53054DF4FF530E517B40A1CAF30EFC470
:10026A00135401F45401FFC43354E0FFE53054DF62
:10027A004FF530051DE4F517E4F552E55213131353
:10028A00541F2412F8E6FD7C00E5525407FF74015E
:10029A007E00A807088005C333CE33CED8F9FFEE17
:1002AA005CFEEF5D4E6043E55225E025E0246EF5E5
:1002BA0082E43400F583E0FEA3E0FFE55225E02561
:1002CA00E0246CF582E43400F583E0FCA3E0C39FEC
:1002DA00EC9E5016E55225E025E0246CF582E434C4
:1002EA0000F583E475F001120649E55225E025E0A0
:1002FA00246EF582E43400F583E0FEA3E0FFE552C4
:10030A0025E025E0246CF582E43400F583E0FCA3C3
:10031A00E0C39FEC9E407AE55225E025E0246CF587
:10032A0082E43400FEC3E582946CFFEE9400FE7C06
:10033A00007D021206137C007D021206137C007DEA
:10034A0008120613741E2FF8C000E6FFC007E55214
:10035A0025E025E0246CF582E43400FEC3E58294AE
:10036A006CFFEE9400FE7C007D021206137C007D79
:10037A00021206137C007D08120613AF057401A849
:10038A0007088002C333D8FCFED0E04ED000F680C6
:10039A0079E55225E025E0246CF582E43400FEC3B9
:1003AA00E582946CFFEE9400FE7C007D0212061337
:1003BA007C007D021206137C007D08120613741E4F
:1003CA002FF8C000E6FFC007E55225E025E0246CBF
:1003DA00F582E43400FEC3E582946CFFEE9400FEDD
:1003EA007C007D021206137C007D021206137C003B
:1003FA007D08120613AF057401A807088002C333EB
:10040A00D8FCF4FED0E05ED000F60552E552642036
:06041A00600302028522CE
:10095D00E51DB41E19AF30EFC413135401F4540147
:10096D00FFC4333354C0FFE53054BF4FF530E51DA0
:10097D00B43C1CAF30EFC413135401F45401FFC445
:10098D00333354C0FFE53054BF4FF530E4F51D222D
:03000B000208B038
:1008B000C0E0C0D075D008758CEEAF30EF131313C5
:1008C0005401F45401FF33333354F8FFE53054F747
:1008D0004FF530053AE53A30E0020516E53AB40A3C
:1008E00015AF30EFC45401F45401FFC454F0FFE5D8
:1008F0003054EF4FF530E53AB4141AAF30EFC4542A
:1009000001F45401FFC454F0FFE53054EF4FF530CB
:0A091000052E753A00D0D0D0E03279
:10091A007594FF752F05E4F530F53190000CF0A3BE
:10092A00F090010BE054F7F054EFF054DFF054BFAD
:10093A00F0547FF090010AE054F7F054EFF054DFDE
:10094A00F054BFF0547FF0A3E054FEF054FDF0548D
:03095A00FBF0228D
:040D9F00752F092281
:10099D00E4FFEF25E025E0246CF582E43400F583D7
:1009AD00E4F0A3F00FBF20EAE4FF7F4090002CE4B9
:1009BD00F0A3DFFCE4FF741E2FF8E4F60FBF04F67E
:0D09CD00E4FF74192FF8E4F60FBF04F622C2
:0E0C9E00758911D2B4D2B9D2A9D28CD2AF22AC
:1009DA00AFA0EFC3135455FEEF25E054AA4EFF1300
:1009EA00135433FEEF25E025E054CC4EFF54F0FEBD
:1009FA00E590540F4EF4F522EF540FF4540FF523FB
:0D0A0A00120A17EFF4F5248528800204205D
:1007BD00E4FF74222FF8E6FE743F2FF8A6060FBF54
:1007CD0006F0E4FF74282FF8E6FE74452FF8A60610
:1007DD000FBF06F0E4FF74682FF8E6FE74202FF5C6
:1007ED0082E43401F583EEF00FBF20EAE4FF74ECF0
:1007FD002FF582E43400F583E0FE74402FF582E49A
:10080D003401F583EEF00FBF20E4E4FF741E2FF8E2
:10081D00E6FE74362FF8A6060FBF04F0E4FF741938
:0F082D002FF8E6FE74322FF8A6060FBF04F02254
:100A760075510112091A12099D120C9E1209DA12F9
:100A8600000E12023A12095D1207BDE55160EDE44F
:070A9600F551120D9F80E5F0
:10000E00AF2F120C45E51130E00790010BE054F7CD
:10001E00F0E51130E00790010BE0547FF0E5113070
:10002E00E04EE490002CF0A3F0FFFEFC7D021206E1
:10003E00137C007D0812061374192FF8C000E6FF1A
:10004E00C007C3742C942CFF74009400FE7C007DBA
:10005E00021206137C007D08120613AF057401A868
:10006E0007088002C333D8FCF4FED0E05ED000F661
:10007E00E5225401FF120C4B90010BE0FFC4131349
:10008E00135401FF120D97E51120E003020169E5FB
:10009E003B30E00302016F4401F53BC390002DE0BD
:1000AE00941490002CE09400400302016FA3E0042E
:1000BE00F0700690002CE004F0C390002DE0941434
:1000CE0090002CE094004049E4FFFEFC7D021206F5
:1000DE00137C007D0812061374192FF8C000E6FF7A
:1000EE00C007C3742C942CFF74009400FE7C007D1A
:1000FE00021206137C007D08120613AF057401A8C8
:10010E0007088002C333D8FCFED0E04ED000F68044
:10011E0050E4FFFEFC7D021206137C007D081206E1
:10012E001374192FF8C000E6FFC007C3742C942C6B
:10013E00FF74009400FE7C007D021206137C007D8D
:10014E0008120613AF057401A807088002C333D83E
:10015E00FCF4FED0E05ED000F68006E53B54FEF5E2
:10016E003BE5195401FF120C4BE51130E0079001ED
:10017E000BE04408F0E51130E00790010BE0547FEE
:10018E00F0AF22120C45E51130E00790010BE05460
:10019E00F7F0E51130E04EE490002CF0A3F0FFFEF6
:1001AE00FC7D021206137C007D0812061374192FB3
:1001BE00F8C000E6FFC007C3742C942CFF740094A3
:1001CE0000FE7C007D021206137C007D08120613D1
:1001DE00AF057401A807088002C333D8FCF4FED023
:1001EE00E05ED000F6AF24EFC3120C47E51130E00D
:1001FE000790010BE04480F0E5245401FF120C4BF4
:10020E00E51130E00790010BE0547FF0E52F54012B
:10021E00FF120C4BE51130E01190002CE0FEA3E034
:0C022E00FF7B017A00790C1207360022D9
:03000000020D1DD1
:0C0D1D00787FE4F6D8FD758187020A7625
:10060100EF8DF0A4A8F0CF8CF0A428CE8DF0A42E0D
:02061100FE22C7
:10061300C2D5EC30E709B2D5E4C39DFDE49CFCEE02
:1006230030E715B2D5E4C39FFFE49EFE1206E1C393
:10063300E49DFDE49CFC80031206E130D507C3E48E
:060643009FFFE49EFE2271
:10064900C5F0F8A3E028F0C5F0F8E582158270023C
:060659001583E038F022D9
:10065F00BB010A89828A83E0F5F0A3E02250068766
:10066F00F009E71922BBFE07E3F5F009E319228928
:0B067F00828A83E493F5F0740193225B
:10068A00BB010789828A83020649500B09C5F027F4
:10069A00F7C5F01937F722BBFE0D09F8E325F0F389
:1006AA00C5F019E338F322F889828A837401932505
:0806BA00F0C5F0F8E4933822CA
:1006C200BB010A89828A83F0E5F0A3F0225006F783
:0F06D20009A7F01922BBFE06F3E5F009F3192280
:1006E100BC000BBE0029EF8DF084FFADF022E4CCFD
:1006F100F875F008EF2FFFEE33FEEC33FCEE9DECC6
:10070100984005FCEE9DFE0FD5F0E9E4CEFD22ED0B
:10071100F8F5F0EE8420D21CFEADF075F008EF2F55
:10072100FFED33FD4007985006D5F0F222C398FD46
:050731000FD5F0EA22E3
:00000001FF
